:100000000C94C5010C94FD010C94FD010C94E11AB3
:100010000C94FD010C94FD010C94FD010C94FD0168
:100020000C94FD010C94FD010C9413220C94E52218
:100030000C94EB1C0C94FD010C94FD010C94FD013F
:100040000C94FD010C94FD010C94FD010C94FD0138
:100050000C94FD010C948F1D0C94FD010C94FD017A
:100060000C94FD010C94FD010C94FD010C94FD0118
:100070000C94FD010C94FD010C94FD010C94FD0108
:100080000C94FD010C94FD010C94FD010C94FD01F8
:100090000C94FD010C94FD010C94FD010C94FD01E8
:1000A0000C94FD010C94FD010C94FD01AD04AD0414
:1000B000D904D90441055F05770677066A0503066A
:1000C0001406140652237923712479237124C5233D
:1000D000E82371243F244E2414001A000800150060
:1000E0001700000004001600070009000A000000C5
:1000F0001D001B000600190005000000E000E100E3
:100100002B00E30001512C00130012000C0018001A
:100110001C00000033000F000E000D000B0000005B
:10012000380037003600100011000000E400E50040
:100130002A00E600025128001E001F0020002100B6
:100140002200000044004A004E004B004D00000019
:100150003A003B003C003D003E000000E000E100B2
:100160002900E30001002C002700260025002400C0
:100170002300000045004F005200510050000000D5
:1001800043004200410040003F0000004600E500FF
:100190004C00E600035128001E021F02200221022B
:1001A00022020000000000000000310035000000C5
:1001B000000000000000310235020000E000E10014
:1001C0002900E30003512C00270226022502240205
:1001D0002302000030022F0234002E002D00000008
:1001E00030002F0034022E022D020000E400E50052
:1001F0004C00E60001002800A900005C000000009F
:1002000000000000AA00C35CC65CC85CCA5C0000B9
:10021000A800C45CC75CC95CCB5C000000000000A7
:100220000000000001000000BD0000000000000010
:1002300000000000BE000000000000000000000000
:1002400000000000000000000000000000000000AE
:10025000000000000100000014037300630061004F
:1002600074007400650072003400320000000E0358
:1002700062006200720066006B00720000000403FE
:10028000090409023B00020100A0FA090400000170
:10029000030101000921110100012240000705812D
:1002A00003080001090401000103000000092111F5
:1002B000010001227B0007058203200001120100DA
:1002C0000200000008EDFE473B01000102000105AD
:1002D000010902A10185020901A1000509190129ED
:1002E00008150025019508750181020501093009ED
:1002F000311581257F9502750881060938158125FC
:100300007F950175088106050C0A38021581257F45
:10031000950175088106C0C005010980A10185030A
:1003200019012AB700150126B70095017510810043
:10033000C0050C0901A101850419012AA0021501BB
:1003400026A002950175108100C005010906A101D2
:10035000050719E029E715002501950875018102B7
:100360009501750881010507190029FF150026FF71
:100370000095067508810005081901290595057580
:10038000019102950175039101C011241FBECFEFA9
:10039000DAE0DEBFCDBF04B603FE18C0809198023C
:1003A00090919902A0919A02B0919B028730904B54
:1003B000A740B04B59F410929802109299021092F3
:1003C0009A0210929B02E0E0F8E3099511E0A0E0A8
:1003D000B1E0EEE7FAE402C005900D92A03AB10751
:1003E000D9F722E0A0EAB1E001C01D92A839B20716
:1003F000E1F70E9452150C943D250C94000081E019
:10040000089581E008950C94010208950C9405026A
:100410001F93CF93DF9300D000D01F92CDB7DEB7EC
:1004200049835A836B833091A30189819A81311169
:1004300014C0662359F0222349F00E94B608182FF1
:10044000682F89819A810E945D0803C00E948908F3
:10045000182F69817A81812F04C00E94B6086981B2
:100460007A810F900F900F900F900F90DF91CF91A6
:100470001F910C94DF0FFC01262F40815181628176
:10048000738184810C94080281E00895CF93DF93F7
:10049000EC0160E00E943B02BE01DF91CF910C9421
:1004A00006020C9463110C945F1108950E940707D3
:1004B0000E9455022FEF84E39CE021508040904041
:1004C000E1F700C000000C94B51D0F931F93CF936C
:1004D000DF938C0161E00E943B02EC01B8010E94B5
:1004E00003028823F1F1B801CE010E94EC198823A0
:1004F000C1F1B801CE010E940018882391F1B80122
:10050000CE010E944819882361F1F8018281882375
:1005100009F1CB358DE5D807C1F050F4C115FCE5E4
:10052000DF0781F0CF3DDC45A9F40E94ED0D19C035
:10053000CC35EDE5DE0761F0CD35DD4559F40E949F
:10054000300D08C00E9456020CC00E94390D02C036
:100550000E943C0DC801DF91CF911F910F910C9427
:10056000FF0180E0DF91CF911F910F9108950E94CC
:10057000CE1C0C94D0020E94D3020C94D41C08957B
:100580000C94BF0281E008950C94C2020895CF93A9
:10059000C82F0E94C0028C2F0E94C402CF910895E0
:1005A00080E00C94C7020E940C1C0C94C7020E94AD
:1005B0000C1C9091A201891721F08093A2010C9448
:1005C000C7020895CF93DF93CDB7DEB72B970FB651
:1005D000F894DEBF0FBECDBF4F83588769877A87F7
:1005E0008B8761110E947C0C9E012F5F3F4F86E03C
:1005F000F90111928A95E9F785E0FE013796D90154
:1006000001900D928A95E1F789819A814C815D81F3
:10061000452B31F09F3F31F491E08F3F19F403C037
:1006200091E001C090E090FF09C049815A816B813F
:100630007C818D819E810E949D0B05C0C9010E9415
:1006400044028111F2CF2B960FB6F894DEBF0FBE95
:10065000CDBFDF91CF910895FC01808191810E94EF
:10066000F8080895CF93882309F4A4C0C82F8238CE
:10067000C1F40E940C1C81FD9DC069E380910201C0
:10068000909103010E94A61C0E949E0C2FEF81EE08
:1006900094E0215080409040E1F700C0000069E301
:1006A00019C0833801F50E940C1C80FD83C063E5EE
:1006B00080910201909103010E94A61C0E949E0C51
:1006C0002FEF81EE94E0215080409040E1F700C090
:1006D000000063E580910201909103010E94A81C33
:1006E000CF910C949E0C8438C1F40E940C1C82FDA6
:1006F00061C067E480910201909103010E94A61CF1
:100700000E949E0C2FEF81EE94E02150804090409B
:10071000E1F700C0000067E4DDCF8CEF8C0F813A79
:10072000D0F46C2F80910201909103010E94701C03
:10073000882349F06C2F80910201909103010E945F
:10074000A81C0E949E0C6C2F8091020190910301C5
:100750000E94A61CC5CF80E28C0F883048F4C77079
:1007600081E001C0880FCA95EAF70E945F0CB8CFFC
:10077000EBE5EC0FE33040F4F0E0E05AFE4F80810F
:1007800090E0CF910C94381CE8E5EC0FE73150F481
:10079000F0E0EE0FFF1FEE5CFE4F80819181CF9164
:1007A0000C944E1CCD3E30F08C2F0E94D715CF916B
:1007B0000C94A916CF910895882309F464C0823857
:1007C00079F40E940C1C81FF5EC069E380910201F4
:1007D000909103010E94A61C0E949E0C69E310C028
:1007E0008338B1F40E940C1C80FF4DC063E58091FA
:1007F0000201909103010E94A61C0E949E0C63E5D9
:1008000080910201909103010E94A81C0C949E0CFF
:10081000843879F40E940C1C82FF35C067E4809113
:100820000201909103010E94A61C0E949E0C67E4A5
:10083000E7CF9CEF980F913A10F4682FE1CF90E248
:10084000980F983050F4877091E001C0990F8A9505
:10085000EAF7892F0E94650CD9CF9BE5980F93305A
:1008600020F480E090E00C94381C98E5980F9731C4
:1008700020F480E090E00C944E1C8D3E20F00E940D
:1008800032160C94A91608951F93CF93DF93182F57
:10089000EB010E943203209741F08FE99FE001971E
:1008A000F1F700C000002197F6CF812FDF91CF91A3
:1008B0001F910C94DC03893319F060E070E002C0F2
:1008C00060E570E00C944404882321F00E945F0CE2
:1008D0000C949E0C0895882321F00E94650C0C94C2
:1008E0009E0C0895CF92DF92EF92FF920F931F9389
:1008F000CF93DF937C01D62FC72FFC011281058196
:1009000002950F700E94550C8823B9F01123A9F0AD
:100910008C2F807F803421F080E28D0F883068F04A
:100920008091740282FD09C082E00E94FE0C0E9448
:10093000550C91E0D82ED92601C0D12CCC2EC294D2
:100940008FE0C8228C2D90E08C30910508F0CFC14B
:10095000FC01EA5AFF4F0C94CB248C2F807FCF7080
:10096000882311F0C295C07F112399F0CC2309F49C
:10097000AAC180E28D0F883010F0D11104C08C2FF5
:100980000E945F0C03C08C2F0E946F0C0E949E0C73
:100990009AC18D2F0E94DC03CC2309F4A8C180E208
:1009A0008D0F883038F1DD2329F18C2F0E94750CD2
:1009B00024C08C2F807FCF70803211F0C295C07F11
:1009C000DD2319F0D130A1F13DC08091740282FF86
:1009D00017C0112349F0CC2329F08C2F0E945F0C03
:1009E0000E949E0C80E070C180E00E94DC03CC235A
:1009F00009F47DC18C2F0E94650C0E949E0C77C16A
:100A0000112371F0002341F0013031F40E947F0C7A
:100A10008C2B0E94870C6BC10E947F0C8C2B1DC0FD
:100A2000002319F0013009F462C10E94940C25C022
:100A3000112321F0063008F05AC10EC0053008F02D
:100A400056C11BC0112361F0002331F0F7018581ED
:100A500080FF39C18F7085838C2F0E94640447C149
:100A6000002359F0D93309F03FC1FFEF07EE13E03F
:100A7000F15000401040E1F735C18C2F0E946B040B
:100A800036C18C2F86958695837019F0813061F080
:100A90002EC1112321F08D2F9C2F937002C080E076
:100AA00090E00E94381C2BC1112321F08D2F9C2F28
:100AB000937002C080E090E00E944E1C20C18D2FF8
:100AC000112319F00E94D71502C00E9432160E940D
:100AD000A91615C18C2F837009F047C011110BC1E5
:100AE0002D2F229526952770220F220F6D2F6F70C4
:100AF000862F90E0A0E0B0E0022E04C0880F991F7E
:100B0000AA1FBB1F0A94D2F7D4FF10C04FE050E0D9
:100B100060E070E004C0440F551F661F771F2A95E0
:100B2000D2F7409550956095709503C040E050E035
:100B3000BA01C695C695C3708A019B01082B192B73
:100B40002A2B3B2BC901B801C23049F058F4C130FF
:100B500019F00E947307CFC00E946107CCC00E94A9
:100B60008507C9C00E945F07C6C0112319F08C2FEA
:100B7000817001C08695882309F4BDC02D2F229570
:100B800026952770220F220F6D2F6F70862F90E011
:100B9000A0E0B0E0022E04C0880F991FAA1FBB1F5F
:100BA0000A94D2F7D4FF10C04FE050E060E070E04C
:100BB00004C0440F551F661F771F2A95D2F7409532
:100BC00050956095709503C040E050E0BA01C6951D
:100BD000C695C3708A019B01082B192B2A2B3B2B2E
:100BE000C901B801C23049F058F4C13019F00E946F
:100BF000380881C00E9426087EC00E944A087BC037
:100C00000E94990778C0CF70112339F08C2F0E9471
:100C1000BF078D2F0E9464046EC08D2F0E946B044D
:100C20008C2F0E94E00767C0D23F21F128F4D03F0B
:100C300041F0D13FC1F043C0D33F19F1D43F79F027
:100C40003EC0112341F0053008F051C08C2F8F7148
:100C50000E9405084CC0063008F049C0F7CF8091CB
:100C6000740282FF18C0112339F08C2F8F710E94FB
:100C7000BF073DC01123C9F38C2F8F710E94E0077D
:100C800036C0112329F08C2F8F710E94AA072FC024
:100C90000E94A5072CC0112349F0CF718C2F0E9410
:100CA000BF0763E08C2F0E94E30C21C081E00E940B
:100CB000FE0C0230E0F082E00E94FE0C18C011230E
:100CC00031F0002391F28D2F0E94320310C00023D7
:100CD00099F2D93349F41FEF27EE33E01150204049
:100CE0003040E1F700C000008D2F0E94DC0388EF48
:100CF0008C0D843020F40E940C1C0E94C702DD2061
:100D0000C9F00E94510C80FD15C0F70112820E94AB
:100D10004B0C0E94BF07C7010E94BB060E944B0CF0
:100D2000DF91CF911F910F91FF90EF90DF90CF90C7
:100D30000C94E007DF91CF911F910F91FF90EF90FE
:100D4000DF90CF9008950F931F93CF93DF93EC0123
:100D5000688179818A810E9403098C010E945C0864
:100D60000E944D07B801CE010E947204DF91CF911D
:100D70001F910F910895CF93DF93EC0198818981A2
:100D80002B813C81232B31F08F3F31F481E09F3F59
:100D900019F403C081E001C080E080FD1DC0CE01D8
:100DA0000E946502811110C00E94550C8823A1F099
:100DB0008A81882389F08091740282FD0DC082E0CF
:100DC000DF91CF910C94FE0CCE010E94A306CE01C0
:100DD000DF91CF910C944602DF91CF91089580E08E
:100DE00090E00E94381C80E090E00E944E1C0E941F
:100DF0007C0C0E949E0C0E94DA170C94A91680911C
:100E00000201909103010E94AA1C0C94EF060E941B
:100E10006C0C0C94FF0692959F70963079F010F44C
:100E2000925001C09A50923068F4803F69F018F4F3
:100E3000883E40F409C0843F29F406C0883E20F073
:100E4000813F11F080E0089581E00895FC018081E8
:100E500091810E94F8080E940B070895CF93DF93B9
:100E600000D000D01F92CDB7DEB70F900F900F903B
:100E70000F900F90DF91CF910895CF93DF9300D023
:100E800000D000D0CDB7DEB726960FB6F894DEBFFF
:100E90000FBECDBFDF91CF910895089508950C94B2
:100EA0004E070C944F070E9451076093C601709340
:100EB000C7018093C8019093C9010C94EF060C946C
:100EC00053070F931F930091C6011091C701209102
:100ED000C8013091C901602B712B822B932B1F917C
:100EE0000F910C9453070F931F930091C60110911B
:100EF000C7012091C8013091C90160237123822369
:100F000093231F910F910C9453070F931F930091FC
:100F1000C6011091C7012091C8013091C901602715
:100F20007127822793271F910F910C9453070C94DC
:100F30004E070E9497076093C2017093C30180938C
:100F4000C4019093C5010C94EF0660E070E0CB0102
:100F50000C9499070F931F9341E050E060E070E01C
:100F60008A019B0104C0000F111F221F331F8A95A5
:100F7000D2F7C901B8011F910F910C9499070F93F3
:100F80001F9341E050E060E070E004C0440F551F43
:100F9000661F771F8A95D2F78091C2019091C30195
:100FA000A091C401B091C5018A019B01082B192BA6
:100FB0002A2B3B2BC901B8011F910F910C94990763
:100FC0000F931F9341E050E060E070E004C0440FD5
:100FD000551F661F771F8A95D2F7409550956095EB
:100FE00070958091C2019091C301A091C401B0910C
:100FF000C5018A019B01082319232A233B23C90128
:10100000B8011F910F910C9499070F931F9341E022
:1010100050E060E070E004C0440F551F661F771F6A
:101020008A95D2F78091C2019091C301A091C40129
:10103000B091C5018A019B01082719272A273B2760
:10104000C901B8011F910F910C9499070F931F9339
:101050000091C2011091C3012091C4013091C501DA
:10106000602B712B822B932B1F910F910C9499075E
:101070000F931F930091C2011091C3012091C401ED
:101080003091C50160237123822393231F910F9117
:101090000C9499070F931F930091C2011091C30103
:1010A0002091C4013091C5016027712782279327C1
:1010B0001F910F910C9499070895292F220F920FD9
:1010C000990F890FE82FE695E695E695877051E030
:1010D00001C0550F8A95EAF785E0E89FF0011124D9
:1010E000EC55FE4F20E030E070E04081CB01022E55
:1010F00002C0969587950A94E2F7817081958427BE
:101100008523842781932F5F3F4F2530310569F771
:101110000895292F220F920F990F890F682F669536
:1011200066956695982F977085E0689FB0011124A9
:1011300040E050E080E0FB01E40FF51FEC55FE4F6E
:10114000208130E0092E02C0369527950A94E2F7F7
:1011500021703327042E01C0220F0A94EAF7822B54
:101160004F5F5F4F4530510531F70895BF92CF92E1
:10117000DF92EF92FF920F931F93CF93DF938C0137
:10118000C090C201D090C301E090C401F090C501AD
:101190008091C6019091C701A091C801B091C90189
:1011A000C82AD92AEA2AFB2ACFE1D0E0D701C60112
:1011B0000C2E04C0B695A795979587950A94D2F7FB
:1011C00080FD04C0219790F7B12C07C0BC2EB80158
:1011D0008C2F0E94F20F0197A9F38B2DDF91CF91F5
:1011E0001F910F91FF90EF90DF90CF90BF900895E7
:1011F000CF93DF93EC010E94B608BE010E94F20F6C
:10120000DF91CF9108951F93CF93DF93EB019091DE
:10121000A301992321F0CB010E94F80813C0882371
:1012200049F0CB010E94B608182F682FCE010E940A
:101230005D0804C0CB010E948908182FBE01812FD0
:101240000E94F20FDF91CF911F9108951F93CF93CA
:10125000DF93C091CA0116E08091CB01C81799F0C5
:10126000D0E01C9FF0011D9FF00D1124E453FE4FB0
:101270004081518162817381848195810E943D0703
:101280002196C770E9CFDF91CF911F9108954091CA
:10129000FC015091FD016091FE017091FF01809170
:1012A0000002909101020C943D07EF92FF920F9380
:1012B0001F93CF93DF938091010282958F7009F085
:1012C00065C08091FE01882309F460C08091CA0145
:1012D000F090CB011091FC010091FD016091FF01A4
:1012E0007091000291E01F3F09F090E0C091000171
:1012F000D0910101292F96E0E92E8F1509F446C0FF
:101300006115710521F00F3F21F030E003C031E09D
:1013100001C0322F90E030FD36C0E89EF001E99E1A
:10132000F00D1124DF01A453BE4F11963C9111978B
:10133000301329C03C91311326C012963C9112976C
:10134000311121C013964D915C911497461B570B98
:101350004C175D07C0F4809101028F70806180930B
:101360000102EF52FE4F80818F70806180838CEF8D
:1013700091E00E94BB06DF91CF911F910F91FF90EA
:10138000EF900C94260901968770B7CFDF91CF912B
:101390001F910F91FF90EF9008959F92AF92BF928F
:1013A000CF92DF92EF92FF920F931F93CF93DF9331
:1013B000CDB7DEB761970FB6F894DEBF0FBECDBFD5
:1013C0008C0185E0F801DE011D9601900D928A9551
:1013D000E1F7D8011296EC909091FC01E091FD01AB
:1013E0002091FF01309100022115310531F0EF3FCE
:1013F00031F481E09F3F19F403C081E001C080E037
:10140000B82FB1709B2E80FD47C1D8014C91119629
:101410005C9111971396AD90BC9014978CEFC82EE9
:1014200081E0D82EF090FE01B501621B730B209174
:10143000000130910101FF2009F4D9C0809101021F
:101440006217730708F095C0282F207F09F052C05B
:101450005E1313C0491311C0FE2CE1100EC08F7033
:101460008061809301020E944709C6010E94BB0669
:1014700080910102F80185834DC1AB2831F05F3FB7
:1014800031F481E04F3F19F403C081E001C080E0F6
:1014900080FD03C081E08E2502C080E090E0F82F3F
:1014A000F170FF2E80FF1CC08091CA012091CB01FA
:1014B00036E0821709F40BC190E0389FF001399FA4
:1014C000F00D1124E453FE4F6181561306C0608174
:1014D000461303C06281E61203C001968770E9CF0C
:1014E000FE2CEE2009F416C18091010281608093E8
:1014F000010254C05E1306C0491304C0E11002C0CB
:10150000F80199C0C8010E942607882361F1EE20E6
:1015100051F120910102822F82958F7090E0029705
:1015200074F08091FC019091FD0198878F8319865A
:10153000BB86AA862C87CE0107960E94BB0686E052
:10154000F801ACEFB1E001900D928A95E1F70E94AD
:1015500055090E9447090AC05E1711F1C8010E948F
:10156000260781112CC0C8010E94BB06FF24F394FA
:10157000D1C0282F207F81F77A2DB98AA88A6E2DB5
:1015800089890E942E078CEF91E00E94BB0686E0BD
:10159000D6011D928A95E9F70E944709F12CBAC03D
:1015A0004913DCCFE110DACFF8018583C8010E942E
:1015B000BB0686E0D6011D928A95E9F7ABC0EE2006
:1015C00091F220910102822F82958F7090E0029714
:1015D0000CF4B5CF8091FC019091FD019A83898331
:1015E0001B82BD82AC822E83CE010196A6CF6217EC
:1015F000730708F044C0FE2CEE2009F4B4CF5E134C
:1016000030C049132EC02091010220FD21C0822F3D
:1016100082958F70482F50E041155105C9F0F801AF
:1016200025834F30510541F08F5F982F9295907F21
:10163000822F8F70892B8583C8010E94BB0686E0AC
:10164000F801ACEFB1E001900D928A95E1F73CC052
:1016500086E0F801ACEFB1E001900D928A95E1F7D8
:1016600059C0C8010E942607811169CF80910102EB
:10167000816080930102C8010E94BB064BC07A2D95
:10168000B98AA88A6E2D89890E942E0786E0D60124
:101690001D928A95E9F718C0EE2009F464CFC801BD
:1016A0000E942607F82E882309F45DCF86E0F80112
:1016B000ACEFB1E001900D928A95E1F78CEF91E0EB
:1016C0000E942C030E9455090E94470923C04D87A0
:1016D0005E878D859E850E94F808292F22952F70A0
:1016E000223028F49F7039F0811105C00BC02430DE
:1016F00028F49F7049F4805E883020F0C8010E9471
:10170000BB069F2CF92C06C0D80115969C91907FA2
:1017100091F7F8CF8F2D61960FB6F894DEBF0FBE0C
:10172000CDBFDF91CF911F910F91FF90EF90DF9090
:10173000CF90BF90AF909F9008951F93CF93DF936A
:10174000CDB7DEB72C970FB6F894DEBF0FBECDBF76
:101750004F83588769877A878B879C87CE01079646
:101760000E94CD098823D1F09F8188852A853B85F9
:10177000232B31F08F3F31F481E09F3F19F403C0F8
:1017800081E001C080E080FD47C04F8158856985B8
:101790007A858B859C850E943D073EC086E0FE01D0
:1017A0003796DE01119601900D928A95E1F7FF813F
:1017B000E8856A857B856115710531F0EF3F31F46D
:1017C00081E0FF3F19F403C081E001C080E080FDAB
:1017D00023C02091CB0130E0C90101968770992781
:1017E0004091CA0150E084179507F1F1F983EA832B
:1017F0007D836C8396E0929FD001939FB00D11245E
:10180000A453BE4FFE01319601900D929A95E1F7D7
:101810008093CB010E94260916E08091CA01909125
:10182000CB01891771F1189FC001112484539E4F79
:101830000E94CD09882329F1E091CA011E9FF00181
:101840001124E453FE4F4081518162817381848170
:1018500095810E943D078091CA0190E001968770B2
:1018600099278093CA01D9CF0E9407071092CB0114
:101870001092CA01ECEFF1E086E0DF011D928A953B
:10188000E9F72C960FB6F894DEBF0FBECDBFDF91FF
:10189000CF911F91089580910A0285958595859530
:1018A000089580910A028770089590910A029770B6
:1018B00081E009F480E008958091150208959091E7
:1018C0001502892B80931502089580959091150239
:1018D000892380931502089510921502089590911E
:1018E0001402892B8093140208958095909114021C
:1018F0008923809314020895109214020895809110
:101900000B02089508950C94820C0C94830C909112
:10191000740292FD08C090910B02981721F08093F9
:101920000B020C94850C089580910B02882329F0FA
:1019300010920B0280E00C94850C0895CF93DF93F6
:10194000E0910201F0910301809115028083E09102
:101950000201F0910301908180911402892B808310
:1019600080910B02882381F0E0910201F091030144
:101970009081892B808380910201909103010E94C4
:10198000641C81110E94940CC0910201D09103014A
:1019900048E050E062E072E0CE010E94E524892B2D
:1019A00069F088E0FE01A2E0B2E001900D928A9514
:1019B000E1F7CE01DF91CF910C941F1CDF91CF9105
:1019C00008950C94820C9091740292FD10C098E0DE
:1019D000899F90011124262B20930A020E94BF07A1
:1019E00080910A028595859585950C94E10C0C945F
:1019F000BF0710920A0280E00C94E10C20910A02C9
:101A00008095822380930A02982F977099F430E092
:101A1000482F082E000C550B2417350759F09091CC
:101A2000740292FD07C08595859585950E94E00713
:101A30000C94F90C08959091740292FB222720F9DE
:101A4000281769F080FB92F99093740280917302D9
:101A5000909174020E94690D82E00C94FE0C08952E
:101A60008091740282FB882780F991E089270C9489
:101A70001B0D81E00C941B0D80E00C941B0D6FEF8F
:101A80007FEF80E090E00C94272580E090E00E94BA
:101A9000032521E0893E9E4F09F020E0822F089522
:101AA00082E090E00C94FB2483E090E00C94FB2413
:101AB000CF9384E090E00E94FB24C82F82E290E064
:101AC0000E94FB242C2F30E0A901582BCA01CF9192
:101AD0000895CF93C92F682F84E090E00E940925D4
:101AE0006C2F82E290E0CF910C940925AB01BC01F0
:101AF0008FE090E00C941B25AB01BC0183E190E0EA
:101B00000C941B2560E070E0CB010C947C0D60E030
:101B100070E0CB010E94760D0C94820D69EE7EEF91
:101B200080E090E00E94272560E082E090E00E9443
:101B3000092560E083E090E00E9409251092C6012B
:101B40001092C7011092C8011092C90160E084E0B0
:101B500090E00E94092560E082E290E00E94092561
:101B600060E085E090E00E94092560E086E090E07A
:101B70000E9409256FEF87E090E00E94092540E070
:101B800050E0BA0188E090E00E941B2560E08DE003
:101B900090E00E94092540E050E0BA0188E190E021
:101BA0000E941B2560E087E190E00E94092540E04B
:101BB00050E0BA018CE190E00E941B2560E070E0EB
:101BC00080E290E00E94272540E050E0BA0188E1E1
:101BD00090E00E941B250C94870D0C948E0D682FAD
:101BE0008EE090E00C9409250E94581D609322021B
:101BF00070932302809324029093250260931E0227
:101C000070931F028093200290932102089585B75C
:101C1000806885BF85B7806885BF08950C941313CD
:101C200008950C94100E0C94100E0C94130E0C943A
:101C3000100E0C94170E0C94100E0E94070E8FE0DD
:101C400091E10E94021C0E941B0E0C94190E0E942E
:101C5000110E0C94100E0E9429110C94C6020E94C1
:101C6000431D0E94CE100E942D130E9464120E94F8
:101C70002B0E0E94E8170E9437130C94150E8F92BA
:101C80009F92AF92BF92CF92DF92EF92FF920F930B
:101C90001F93CF93DF93CDB7DEB72A970FB6F89493
:101CA000DEBF0FBECDBF0E948812982E81110E9408
:101CB000F40D86E1A82E82E0B82E00E010E0802E20
:101CC000802F0E944D11D82EF501C1905F01C826CA
:101CD000B1F40F5F1F4F0830110589F78FEF89832B
:101CE0008A831B820E944C1D8160782F9D838C8388
:101CF00049815A816B818D810E94E2022FC08091BF
:101D0000260281FD0E945311E12CFF24F3948C2DB7
:101D10008F21F1F00E940E0E882399F0EE828F82BF
:101D2000DF2081E009F480E088870E944C1D8160FB
:101D3000782F9A8789874E815F8168858A850E947E
:101D4000E202F801EA5EFD4F8081F826F08206C0CB
:101D5000E394FF0CF6E0EF12DACFBBCF81E09110F5
:101D600001C080E02A960FB6F894DEBF0FBECDBF4B
:101D7000DF91CF911F910F91FF90EF90DF90CF9067
:101D8000BF90AF909F908F9008950E943F0E0E9449
:101D900013130E94C7160C94D702CF93DF930E94AF
:101DA000F70FEC01811521E5920708F045C0811578
:101DB00030E5930708F094C0883E910528F5803EF1
:101DC000910508F0F8C0883A910570F4853A9105BC
:101DD00008F07CC08130910509F475C008F4E8C0B2
:101DE000049708F0E8C0E4C08F3B910508F0E0C01C
:101DF000C85AD0E0CC0FDD1FCD59DE4F0990D881F5
:101E0000C02DCE019464D8C0811540E2940758F4E7
:101E1000811551E0950708F0CEC08D3E910508F47C
:101E2000C7C09065C9C0C11580E4D80708F4C0C018
:101E3000DF70CE01906AC0C0811525E59207A8F435
:101E4000811534E5930708F095C0811543E59407A3
:101E500008F07BC0811552E5950708F061C0D82FC6
:101E6000CC27CE01816F906AA7C0C11589E5D8073C
:101E7000A0F4C11528E5D20708F082C0C11536E5E7
:101E8000D30708F095C08C2F0E948B108F7190E0C3
:101E9000D82FCC27CE0190628FC0C1154AE5D40758
:101EA00008F474C0CE0190568115904208F080C0AD
:101EB0008D2F8F710E948B10DD27D0628F71AE0144
:101EC000582BCA0179C081E090E076C0C55AD0E0B5
:101ED000CF56DE4F8881C82FD0E0CE0190646CC011
:101EE00074E0969587957A95E1F7282F23703C2F1B
:101EF000337081E090E002C0880F991F3A95E2F7B5
:101F00009C68AC01522B9A019C2F9F7096959695D8
:101F100050E2959FE0011124C9018C2B9D2B4CC0F0
:101F20008370992721E030E002C0220F331F8A9589
:101F3000E2F79C2F9695969580E2989FE0011124F8
:101F4000C22BD32BCE019C6837C08370992721E028
:101F500030E002C0220F331F8A95E2F79C2F96953E
:101F6000969540E2949FE0011124C22BD32BCE0121
:101F70009A6822C0D82FCC27CE01846F906A1CC0EB
:101F8000DC2FCC27CE01806F906A16C08C2F8F700B
:101F90000E948B1094E0D695C7959A95E1F7CF7083
:101FA000D0E0DC2FCC27D0699E01282BC90104C0CA
:101FB00080E090E001C0CE01DF91CF91089520E351
:101FC000829FC0011124FC0126E0729FE00DF11DEB
:101FD0001124E60FF11DEE0FFF1FE852FF4F859110
:101FE000949108950E94DF0F0E94CD0E08958238CB
:101FF000910569F1B0F48133910509F46DC048F49D
:102000008932910509F463C08A32910509F469C0E7
:1020100008958533910509F455C089339105B9F0C8
:102020000895833E910569F138F4803E9105B1F041
:10203000823E910509F10895863E9105A9F1873EFA
:102040009105B9F1843E910509F064C023C0209147
:10205000730220FD4FC021FD4DC008958091730291
:1020600080FD44C08091740280FF44C0809173025F
:1020700084FD42C083EE4DC08091730282FF38C060
:10208000F5CF8091730282FD33C08091740280FD90
:1020900031C0ECCF8091740281FF32C08091730215
:1020A00084FD2AC087EE35C08091730283FF26C06D
:1020B000F5CF8091730283FD21C08091740281FD70
:1020C0001FC0ECCF8091730285FD1CC01DC08091A4
:1020D000730285FD19C016C08091730286FD16C07B
:1020E00017C08091730286FD13C010C089E311C030
:1020F00082EE0FC080EE0DC080E00BC086EE09C0FE
:1021000084EE07C089E205C085E303C08AE201C00E
:1021100081E390E008959091730292FF0DC0282F03
:102120002871283019F4877F846006C0282F247115
:10213000243011F48B7F886093FF0DC0282F287105
:10214000283119F4877E846106C0282F2471243138
:1021500011F48B7E88612091740220FF0DC0382F0E
:102160003871383019F4877F816006C0382F31719B
:10217000313011F48E7F886021FF0DC0282F287127
:10218000283119F4877E816106C0282F2171213101
:1021900011F48E7E886194FD877E089510926F02FF
:1021A0001092700210927102109272020895CF92F2
:1021B000DF92EF92FF926B017C010E941313811159
:1021C0000EC00E94581DC61AD70AE80AF90AC09222
:1021D0006F02D0927002E0927102F0927202FF9050
:1021E000EF90DF90CF9008950F931F930E941313E9
:1021F000882321F01F910F910C94581D0E94581DA7
:1022000000916F0210917002209171023091720260
:10221000600F711F821F931F1F910F91089580E01F
:1022200008950C943F0D0E9488128FE39CE901975A
:10223000F1F700C000000E94881280E00E944D115A
:1022400080FF04C00E9411110C94B51D08950C94D8
:1022500013110E94450D811102C00E94ED0D0E94D4
:10226000500D809326020E94580D90937402809323
:1022700073020E9427110E94540D682F70E080E0C5
:1022800090E00E945F076091C2017091C30180914C
:10229000C4019091C5010C949707E82FF0E0E25833
:1022A000FD4F80810895089580EA8A95F1F7089599
:1022B00000C008950C94541108950C945C110C9472
:1022C0005D110C945C110C9461110C945C110F93D2
:1022D0001F93CF93DF9300D000D0CDB7DEB70E941D
:1022E0001313609186028823E9F119821A821B82F6
:1022F0001C82862F90E08E010F5F1F4FB80182581D
:102300009D4F0E944513882389F08091750290E0CB
:1023100044E050E0B80182589D4F0E94E52421E03E
:1023200020932702892B69F410E019C080912702BD
:102330008823D1F384E0F80111928A95E9F710928D
:102340002702E0917502F0E0E258FD4F89819A8101
:10235000AB81BC8180839183A283B38311E00E940F
:1023600053020DC070E062587D4F8091750290E07D
:1023700082589D4F0E94CF130E94651110E0812F5B
:102380000F900F900F900F90DF91CF911F910F91B1
:102390000895F894E82FE295EF70F0E031A1282F2E
:1023A0002F7081E090E001C0880F2A95EAF7982FFE
:1023B0009095932391A392A1892B82A37894089559
:1023C0000F931F93CF93DF93CAE9D1E089918F3F99
:1023D00011F00E94C91181E0CE39D807B9F7C4E9DC
:1023E000D1E00AE911E089918F3F11F00E94C911F3
:1023F0000C171D07C1F7DF91CF911F910F91089521
:10240000CF92DF92EF92FF920F931F93CF93DF93C0
:102410008C01C62FD0E0CE0186569E4F7C01FC0178
:1024200090819F3F09F447C0D62EF894E92FE2959A
:10243000EF70F0E081A19F7021E030E001C0220F39
:102440009A95EAF7822B81A382A12095282322A3C3
:1024500078940E945811E4E9F1E04AE951E031E052
:10246000C12C21912F3F89F0A22FA295AF70B0E02F
:1024700090968C9190E02F7002C0959587952A9543
:10248000E2F780FD02C0832F01C080E0C82A330F2D
:102490004E175F0731F7F70180818F3F11F00E94DF
:1024A000C91161E0C11001C060E08D2D0E945A1178
:1024B000C00FD11FC882DF91CF911F910F91FF9064
:1024C000EF90DF90CF9008958091040180910401F6
:1024D000811102C094E001C090E09093860284E0F4
:1024E000891B809375020E94E01188E0EEE7F2E01C
:1024F000DF01982F1D929A95E9F7E6E7F2E0DF01F8
:102500001D928A95E9F784E00E94DC120C94510236
:10251000EF92FF920F931F93CF93DF93CDB7DEB768
:1025200028970FB6F894DEBF0FBECDBF8E010F5FA8
:102530001F4F88E0F80111928A95E9F7F12C6F2D71
:10254000C8010E940012F394F4E0FF12F8CF48E0B3
:1025500050E0B80186E792E00E94E5247C0121E08A
:10256000892B09F420E0E114F10441F088E0F8013E
:10257000A6E7B2E001900D928A95E1F7609186029C
:1025800070E062587D4F44E086E792E00E94DD12E1
:10259000EF2819F40E94671102C081E090E02896AC
:1025A0000FB6F894DEBF0FBECDBFDF91CF911F9164
:1025B0000F91FF90EF9008950895FF920F931F934E
:1025C000CF93DF938C01F62ED72FC42F222349F00F
:1025D00081E080932A020E944C1D909329028093EF
:1025E000280280912A028823C1F0809128029091CC
:1025F00029020E94641D059780F0EF2DFD2FD80160
:102600004C2F50E0CD01801B910B841795071CF4D3
:102610008D918193F7CF10922A02DF91CF911F9174
:102620000F91FF90089580912D0281110DC00E949D
:10263000AA24811102C082E001C081E080932D02B2
:10264000823011F40E94A52481E090912D029130F6
:1026500009F080E008950C9413130E942B138093CB
:1026600004010E94131381110C947D1308950E949C
:102670001313811102C00C947F13089581E090918F
:102680002E029A3008F080E008950F931F93CF93A5
:10269000DF93EC018B0180912E028A3038F4B8016F
:1026A000CE010E94CD1381111DC00AC080912B0262
:1026B00090912C020E94641D843F914080F715C0C8
:1026C00080912E028F3F19F08F5F80932E028091B0
:1026D0002E028A3060F00E944C1D90932C02809351
:1026E0002B0203C010922E0202C080E001C081E0E4
:1026F000DF91CF911F910F9108950C949B1A0C9428
:102700009E1ADF92EF92FF920F931F93CF93DF9366
:102710007901C82F880FDD0B41155105A9F0FE0185
:1027200093E0EE0FFF1F9A95E1F7EB5FFE4F81817B
:102730009281815D9D4F208130E04217530708F45C
:102740009A01A9010E94F224CE010E94871BD82E73
:102750008823D1F001151105B9F083E0CC0FDD1FFE
:102760008A95E1F7FE01EB5FFE4F438150E00417CD
:10277000150708F4A801CB5FDE4F6C817D81615D98
:102780007D4FC7010E94F2248D2DDF91CF911F91C3
:102790000F91FF90EF90DF9008950C94F0140C943B
:1027A0000C150F931F93CF93DF9300D000D0CDB7BC
:1027B000DEB760914402709145028091460290918B
:1027C00047020E94731D643671058105910528F149
:1027D0000E94F410DC01CB010296A11DB11D89837A
:1027E0009A83AB83BC8300E010E020E030E044E05B
:1027F00050E0BE016F5F7F4F82E00E948113182F6F
:10280000882361F00E94581D609344027093450232
:10281000809346029093470201C011E0812F0F90F0
:102820000F900F900F90DF91CF911F910F9108950E
:10283000AF92BF92CF92DF92EF92FF920F931F93CE
:10284000CF93DF937C015B016A010E943E138111EB
:1028500003C001E010E002C00AE010E0C1E0D0E0F7
:10286000F894B501C701F60109957894811115C056
:1028700021960C171D0794F0CC9F9001CD9F300D31
:10288000300D112480E090E045E34A95F1F7000017
:10289000019682179307C1F7E3CF81E0DF91CF91D3
:1028A0001F910F91FF90EF90DF90CF90BF90AF906E
:1028B0000895AF92BF92CF92DF92EF92FF920F9363
:1028C0001F93CF93DF9300D000D01F92CDB7DEB718
:1028D0005B01E0909E01F0909F0101E010E09E01FD
:1028E0002B5F3F4F40E050E060E070E080E00E94EE
:1028F0008113182F882309F43EC067018FEFC81A8F
:10290000D80A6091400270914102809142029091F8
:1029100043020E94731D643671058105910518F10B
:1029200004E010E09E012F5F3F4F40E050E060E088
:1029300070E081E00E948113182F64E070E0C6010E
:102940000E94E91791E02D81281390E0192351F19D
:102950000E94581D6093400270934102809342028E
:102960009093430211C064E070E0C6010E94E91731
:102970009D818913D5CFF70181819281A381B48193
:1029800089839A83AB83BC83112361F089819A8107
:10299000AB81BC8180933C0290933D02A0933E02A8
:1029A000B0933F0280913C0290913D02A0913E0283
:1029B000B0913F02F50180839183A283B383812F7D
:1029C0000F900F900F900F900F90DF91CF911F916C
:1029D0000F91FF90EF90DF90CF90BF90AF90089550
:1029E0000F931F93CF93DF93EC018B0149E554E1E3
:1029F0000E941814882351F041ED53E1B801CE0133
:102A0000DF91CF911F910F910C94181480E0DF910A
:102A1000CF911F910F9108950F931F93CF93DF9341
:102A2000F894C0919E01D0919F01CE01019624E0BF
:102A3000FB01DC0101900D922A95E1F764E070E062
:102A40000E94E91788837894F8946D817E818F8144
:102A50009885009138021091390220913A02309104
:102A60003B02601771078207930751F060933802A9
:102A70007093390280933A0290933B020E94D710E0
:102A80007894DF91CF911F910F9108950E946B1F51
:102A90000E942F0E0C94771F0E947B1F0E94C50E70
:102AA0000C94951F0E94EA1C0E94521F0E941D0E4A
:102AB0000E9446150E944C150E94270EFBCF809164
:102AC0004E0280FF06C06091220170E0660F771F02
:102AD00026C081FF04C06091220184E005C082FF0E
:102AE00007C06091220188E0689FB001112417C0DF
:102AF00090914D029923D1F060912101961788F7AA
:102B00002091220188E0289F90011124929FA0012A
:102B1000939F500D112470E0CA010E94B7246038C1
:102B2000710540F46115710519F406C068E070E0A4
:102B3000862F08958FE7089581E0089580914E02D1
:102B400080FF08C060911E0170E0759567957595CE
:102B5000679521C081FF06C060911E0170E07595E8
:102B6000679519C082FF04C060911E0170E010C01B
:102B700090914C02992399F060911D019617A0F74E
:102B800080911E01899FC001112470E00E94B7242A
:102B90006038710540F46115710519F406C061E0F3
:102BA00070E0862F08958FE7089581E008958D3EA7
:102BB00021F40E945F15819504C08E3E29F40E9485
:102BC0005F158093520208958F3E21F40E945F1595
:102BD000819504C0803F29F40E945F1580935102C3
:102BE0000895893F19F40E949E1505C08A3F31F46B
:102BF0000E949E1581958093530208958B3F21F486
:102C00000E949E15819504C08C3F29F40E949E1558
:102C10008093540208959FE0980F983078F421E053
:102C200030E0A90102C0440F551F9A95E2F7CA018E
:102C300090915002892B8093500208958D3F21F48A
:102C400080914E0281600BC08E3F21F480914E0234
:102C5000826005C08F3F29F480914E02846080938A
:102C60004E0208958D3E39F49091520297FF35C07F
:102C70001092520259C08E3E29F4909152021916B8
:102C8000BCF32BC0909151028F3E29F497FF25C0D1
:102C90001092510249C0803F19F41916CCF31DC09F
:102CA00090915302893F29F41916BCF410925302F3
:102CB0003BC08A3F19F497FF10C0F8CF8B3F39F41F
:102CC0009091540297FF09C0109254022DC08C3F7E
:102CD00021F4909154021916BCF39FE0980F98309C
:102CE00080F421E030E0A90102C0440F551F9A95FD
:102CF000E2F7CA0180959091500289238093500297
:102D000013C08D3F21F480914E028E7F0BC08E3F09
:102D100021F480914E028D7F05C08F3F29F4809170
:102D20004E028B7F80934E0280915102811106C02A
:102D300080915202811102C010924D028091530283
:102D4000811106C080915402811102C010924C0280
:102D500008950E944C1D20915102211104C0209120
:102D60005202222321F090934B0280934A02209139
:102D70005302211104C020915402222321F0909388
:102D80004902809348028FE492E00C942A1CEF924F
:102D9000FF920F931F93CF93DF9300D000D000D00A
:102DA000CDB7DEB786E0EFE4F2E0DE0111960190E8
:102DB0000D928A95E1F7E0905102F0905202009155
:102DC000530210915402109251021092520210922A
:102DD000530210925402E11003C0FF2009F45DC0B9
:102DE00080914A0290914B020E94641DAC01909127
:102DF0004D02992339F02091230130E02417350743
:102E000058F04BC0209124018AE0289F90011124A2
:102E10002417350718F041C09F3F19F09F5F90932A
:102E20004D02EE2061F00E945F151E1414F09FEF1A
:102E300001C091E0989F902D112490935102FF20A2
:102E400061F00E945F151F1414F09FEF01C091E024
:102E5000989F902D11249093520230915102332368
:102E6000E1F0209152022223C1F045EB3403C0016E
:102E70001124992319F09093510203C081E08093AB
:102E8000510235EB2303C0011124992319F09093CB
:102E9000520203C081E080935202011103C011234A
:102EA00009F45DC080914802909149020E94641D1E
:102EB000AC0190914C02992339F020911F0130E030
:102EC0002417350758F04BC0209120018AE0289F35
:102ED000900111242417350718F041C09F3F19F0C5
:102EE0009F5F90934C02002361F00E949E15101684
:102EF00014F09FEF01C091E0989F902D11249093C2
:102F00005302112361F00E949E15111614F09FEFD9
:102F100001C091E0989F902D11249093540230911C
:102F200053023323E1F0209154022223C1F045EBF8
:102F30003403C0011124992319F09093530203C064
:102F400081E08093530235EB2303C00111249923C0
:102F500019F09093540203C081E080935402809151
:102F6000510281110BC080915202811107C08091E2
:102F70005302811103C08091540281110E94A9164D
:102F8000EB82FC820D831E8386E0FE013196AFE466
:102F9000B2E001900D928A95E1F726960FB6F8946B
:102FA000DEBF0FBECDBFDF91CF911F910F91FF907C
:102FB000EF900895EFE4F2E086E0DF011D928A953C
:102FC000E9F710924D0210924C0210924E020895B1
:102FD0000895FC01680F791F8FEF91E3E617F7075B
:102FE00071F02191822728E030E087FF03C0880F2D
:102FF000892701C0880F21503109B9F7EFCF089513
:10300000CF93DF93EC01FB018281882309F43CC15B
:10301000C430FDE5DF0760F4CB3F9CE5D90788F4B9
:103020009E0122503C452431310508F02EC109C0D3
:10303000C236EDE5DE0729F0C63AFDE5DF0709F007
:1030400024C10E94580D9093740280937302C13181
:103050008CE5D80709F4C6C008F042C0C930ECE5D9
:10306000DE0709F49BC000F5C5308CE5D80709F4EC
:1030700085C078F4C330ECE5DE0709F478C008F0C9
:103080007AC0C230DC4509F0F5C0809173028160DE
:10309000EFC0C7309CE5D90709F478C008F07AC0C2
:1030A000809173028061E4C0CD30FCE5DF0709F454
:1030B00087C058F4CB309CE5D90709F479C008F0F3
:1030C0007BC08091730288606FC0CF30FCE5DF0762
:1030D00009F480C008F082C080917302877FC8C065
:1030E000CE3F9CE5D90709F471C000F5C531FCE578
:1030F000DF0709F485C068F4C3319CE5D90709F4FA
:1031000075C008F095C00E940707809173028F7701
:10311000AFC0CC3FFCE5DF07A9F108F054C0CB3FBE
:10312000DC4509F0A7C08091740240C0C230EDE5D3
:10313000DE0709F489C058F4C1158DE5D80709F4F4
:103140005AC008F069C08091740282602FC0C236F4
:10315000EDE5DE0709F47CC0C63AFDE5DF0709F4BA
:1031600081C0C330DD4509F085C080E06EC080912C
:10317000730282607DC08091730216C080917302D9
:10318000886076C08091740282604FC08091730223
:1031900080626EC08091730280646AC00E940707DB
:1031A00080917302806864C0846062C081603DC0A9
:1031B000809173028E7F5CC0809173028D7F58C0B6
:1031C0008091730216C08091740218C080917402BD
:1031D0008D7F2BC0809173028F7E4AC080917302D5
:1031E0008F7D46C0809173028F7B42C080917302B5
:1031F000877F8B7F3DC0809174028D7F8E7F15C04D
:103200008091730282FB222720F991E0922790FBA4
:1032100082F990FB83F92CC080917402982F9095CD
:1032200091708E7F892B90FB81F98093740222C06C
:103230000E9407078091730287FB222720F991E003
:10324000922790FB87F914C081E00E94EF0D12C015
:103250008091730284FB222720F991E0922790FB52
:1032600084F906C080917302982F909590FB80F9A5
:103270008093730280917302909174020E94690D91
:103280000E94070780E001C081E0DF91CF9108959F
:10329000CF93DF9386319C4541F5EB010E945C0C96
:1032A000982F8A812091020130910301882379F0BF
:1032B0009A7A81E009F480E080935502911102C06E
:1032C00069E201C065E3C9010E94A61C0AC08091A1
:1032D0005502811102C069E201C065E3C9010E9483
:1032E000A81C0E949E0C80E001C081E0DF91CF917C
:1032F00008950F931F93CF93DF93C42FD22FFC0118
:1033000082818823C9F0409358020E944C1D9093FB
:1033100057028093560280E28C0F883008F057C025
:10332000C77081E001C0880FCA95EAF7DF91CF919D
:103330001F910F910C94640480915802481330C07F
:1033400080915602909157020E94641D883C91051D
:1033500038F510E21D0FCD17B9F080E28C0F8830E0
:1033600040F4C77081E001C0880FCA95EAF70E9457
:103370006B04183028F581E09D2F977001C0880FED
:103380009A95EAF70E946404802F0E945B0418302B
:10339000F0F4D77081E001C0880FDA95EAF70AC02F
:1033A00080E28C0F883098F4C77081E001C0880FEC
:1033B000CA95EAF7DF91CF911F910F910C946B049E
:1033C000802FDF91CF911F910F910C945B04DF91BF
:1033D000CF911F910F9108950F939C01CB01243F32
:1033E0004CE5340731F188F4293DFCE53F07D9F07D
:1033F0002A3D4CE5340779F1283D3C45A9F506E224
:1034000021EE41EE68ED7CE52BC0263FFCE53F0751
:10341000E1F0A8F0273F3C4539F507E225EE46EEFE
:1034200067EF7CE51DC007E225EE45EE69ED7CE522
:1034300017C006E221EE40EE64EF7CE511C007E222
:1034400025EE44EE65EF7CE50BC006E221EE42EE90
:1034500066EF7CE505C008E221E045EE6AED7CE51B
:103460000E94791980E008C0FC018281882319F04C
:103470001092580201C081E00F9108958EE14A9B9D
:1034800002C08150E1F74A9BFECF08955A9880E22E
:103490008A95F1F75A9A0895FC012AE02A95F1F7E6
:1034A00028E090E080E031E040E14A95F1F7880FB4
:1034B0004A9B02C08160932700C0000040E14A950A
:1034C000F1F7215089F720E12A95F1F729B100C0E1
:1034D000000030E13A95F1F722FB222720F99227EC
:1034E0002081920F90830895EF92FF920F931F9384
:1034F000CF93DF931F92CDB7DEB719828C017C0189
:10350000E60EF11C0E151F0551F00E943E1ACE0169
:1035100001960E944C1AF80181938F01F3CF81E04C
:103520009981911180E00F90DF91CF911F910F91C0
:10353000FF90EF900895529A5A9A089552985A9A85
:10354000EA9AE9E6F0E080818F7C808308956150FB
:1035500091E001C0990F6A95EAF720E031E09923E4
:1035600061F0492F482319F05A9A232701C05A982D
:1035700040E24A95F1F79695F2CF222311F05A9A3C
:1035800001C05A9880E28A95F1F75A980895FF92FF
:103590000F931F93CF93DF93EC018C01060F111D46
:1035A000C017D10741F0F9900E94461A68E08F2DAC
:1035B0000E94A71AF5CFDF91CF911F910F91FF9035
:1035C00008951F920F920FB60F9211240F931F931D
:1035D0002F933F934F935F936F937F938F939F931B
:1035E000AF93BF93EF93FF93CF93DF931F92CDB72A
:1035F000DEB719820E943E1ACE0101960E944C1A33
:10360000082F069506950695902F96959570202F74
:103610002570920F292F237096959695920F87709B
:1036200089135FC0898181115CC0043008F059C0E2
:1036300080E18A95F1F75A9A529A82E08A95F1F7D9
:1036400000C05A9888E0089F80011124D801AB5F20
:10365000BE4F1696ED91FC9117973097A9F06091A7
:103660009E0170919F0114962D913C911597260F04
:10367000371F11968D919C911297680F791F1396A1
:103680004C9113978C910995F801EB5FFE4F638184
:10369000662351F080919E0190919F012481358194
:1036A000820F931F0E94C71A0E94461A80E18A95D2
:1036B000F1F75A9852985A9A80E18A95F1F7F801F1
:1036C000EB5FFE4F6081662351F080919E019091E7
:1036D0009F0121813281820F931F0E94741A0E94E0
:1036E0003E1A0F90DF91CF91FF91EF91BF91AF9173
:1036F0009F918F917F916F915F914F913F912F910A
:103700001F910F910F900FBE0F901F9018950F9360
:103710001F93CF93DF93843091050CF06DC0EC01C3
:10372000F894529A5A9885E08A95F1F700009C2FF8
:10373000969595702C2F2570920F892F83709695F2
:10374000969523E0CC0FDD1F2A95E1F7980F8E01A7
:10375000092B0E94461A84E08A95F1F700C068E0C0
:10376000802F0E94A71A80E18A95F1F752985A9A01
:103770004A9902C000C0FCCF87E090E04A9B08C095
:10378000019721F4529A5A9A789436C000C0F6CF25
:10379000FE01EB5FFE4F6381662381F080919E0105
:1037A00090919F0124813581820F931F0E94741A8A
:1037B000811104C0529A5A9A78941FC00E943E1AEE
:1037C00080E28A95F1F75A98529A80E18A95F1F74A
:1037D000CB5FDE4F6881662351F080919E0190910E
:1037E0009F0129813A81820F931F0E94C71A0E946C
:1037F000461A789481E001C080E0DF91CF911F915B
:103800000F9108959093A1018093A0010895909342
:103810005F0280935E0208950E941313811103C01A
:10382000809159020895E0915E02F0915F02309715
:1038300021F00190F081E02D099480E00895E0915D
:103840005E02F0915F02309721F00280F381E02D5B
:1038500009940895E0915E02F0915F02309739F08B
:1038600022E0DC012C930480F581E02D0994089579
:1038700020915C0230915D022817390771F0909316
:103880005D0280935C02E0915E02F0915F023097EE
:1038900021F00680F781E02D0994089520915A02C5
:1038A00030915B022817390771F090935B02809387
:1038B0005A02E0915E02F0915F02309721F000849D
:1038C000F185E02D09940895FC01329697E080E09F
:1038D000915029F021912223D9F38F5FF9CF0895D8
:1038E000662349F0FC01329608962191621729F06F
:1038F000E817F907D1F780E0089581E008959C0169
:10390000FC0132969FEF80E04191461789F09F3F7E
:1039100019F4411101C0982F8F5F8630A9F79F3F9E
:1039200039F0F901E90FF11D97FDFA9562830895C9
:1039300008959C012A5F3F4FFC014281461301C05C
:103940001282019682179307B9F708950C947F1C91
:103950000C94991C029626E0FC0111922A95E9F735
:10396000089508950C94B11C83E0809360020C9438
:10397000B21C811102C081E001C082E0809360022C
:103980000C94B21C0C94B91C81E0809360020C94DE
:10399000B21C0C94C41C08950C94CB1C0C94CC1C2D
:1039A0000C94CB1C0C94CB1C0C94CB1CCF930E947E
:1039B000D21C0E9488120E94D01CC0E08C2F0E9452
:1039C0004D11811104C0CF5FC830C1F701C081E043
:1039D000CF91089508951F920F920FB60F92112460
:1039E0008F939F93AF93BF9380916102811113C016
:1039F0008091870290918802A0918902B0918A02F9
:103A00004196A11DB11D8093870290938802A093D7
:103A10008902B0938A02BF91AF919F918F910F90CD
:103A20000FBE0F901F90189580918F02843031F156
:103A30000E94B7021092610220E488E190E00FB684
:103A4000F894A895809360000FBE2093600083B720
:103A5000817F846083BF83B7816083BF78948895BA
:103A600083B78E7F83BF0FB6F894A89580916000CE
:103A7000886180936000109260000FBE08950E94DC
:103A800007070C94BB0282E084BD93E095BD9AEFDA
:103A900097BD80936E0008952FB7F89480918702A8
:103AA00090918802A0918902B0918A022FBF089557
:103AB0002FB7F894609187027091880280918902F3
:103AC00090918A022FBF08959C014FB7F89480917E
:103AD000870290918802A0918902B0918A024FBF1B
:103AE000821B930B0895CF92DF92EF92FF922FB734
:103AF000F894C0908702D0908802E0908902F090FC
:103B00008A022FBFA7019601261B370B480B590BC2
:103B1000CA01B901FF90EF90DF90CF90089578949B
:103B20001F920F920FB60F9211248F939F93AF9312
:103B3000BF938091870290918802A0918902B091F1
:103B40008A020196A11DB11D80938702909388027D
:103B5000A0938902B0938A02BF91AF919F918F91F8
:103B60000F900FBE0F901F90189581E08093E0009A
:103B700080E28093D8001092C9008FE19EE4019703
:103B8000F1F700C0000087E090EBDC018093980221
:103B900090939902A0939A02B0939B029CE088E1D3
:103BA0000FB6F894A895809360000FBE90936000C4
:103BB000FFCF80916D020895089522E02093E900DF
:103BC0002FEF3091E800215035FD06C035ED3A95D4
:103BD000F1F700002111F5CF2091E80025FF0BC07F
:103BE00040E050E066E070E00E9407208091E8002D
:103BF0008E778093E8000895CF93DF9321E02093A0
:103C0000E9002FEF3091E800215035FD06C035ED79
:103C10003A95F1F700002111F5CF2091E80025FF3A
:103C200014C0EC0140E050E068E070E00E94072022
:103C30008091E8008E778093E80088E0FE01A5E699
:103C4000B2E001900D928A95E1F7DF91CF9108954E
:103C500080936202709364026093630280918F028A
:103C6000843001F582E08093E9008FEF9091E800C5
:103C7000815095FD06C095ED9A95F1F700008111F0
:103C8000F5CF8091E80085FF0DC040E050E063E093
:103C900070E082E692E00E9407208091E8008E7733
:103CA0008093E8000895BC0184E00C94281EBC01B8
:103CB00083E00C94281E80918E02811109C00E941D
:103CC00098210E94F5218091E20084608093E200B7
:103CD000089510928E0208950C94C91C60918B0275
:103CE00081E0611101C080E00C94B41C90918F02BE
:103CF00081E0943009F080E060918B020C94B91C53
:103D000042E061EC81E00E94112142E261EC82E03C
:103D10000E94112190918F0281E0943009F080E09F
:103D200060918B020C94C21C80919102833009F443
:103D300061C030F4813071F0823009F49AC0089586
:103D40008A3009F486C08B3009F46CC0893009F0E0
:103D5000A8C020C080919002813A09F0A2C0809151
:103D6000E800877F8093E80080919402909195020B
:103D7000892B21F468E085E692E003C060E080E0F2
:103D800090E070E00E9452208091E8008B77809351
:103D9000E800089580919002813209F082C08091FC
:103DA000940290919502029708F07BC08091E80000
:103DB000877F8093E8008091E80082FD05C08091B4
:103DC0008F028111F8CF6DC02091F3008091F20035
:103DD00090E0922B029731F48091F100813011F044
:103DE000863021F48091F10080936D028091E8008B
:103DF0008B7753C080919002813A09F052C0809134
:103E0000940290919502892B09F04BC08091E800B3
:103E1000877F8093E8008091E80080FFFCCF80914D
:103E2000310136C0809190028132D9F5809194029F
:103E300090919502892BA9F58091E800877F809366
:103E4000E8000E94462180919202809331010C94F7
:103E5000070780919002813221F58091E800877FE9
:103E60008093E8000E9446218091930280936E0225
:103E7000089580919002813AA1F48091E800877FB3
:103E80008093E8008091E80080FFFCCF80916E0273
:103E90008093F1008091E8008E778093E8000C9485
:103EA0004621089584B7877F84BF0FB6F894A895FC
:103EB00080916000886180936000109260000FBE66
:103EC00090E080E80FB6F8948093610090936100D1
:103ED0000FBE0C94C41C0E9498210E94F521E2EEB2
:103EE000F0E080818460808378940C948A2485E259
:103EF00091E00C94071C80918F028530A9F4809189
:103F00008F02853079F40E94141D80918D028823E0
:103F1000B1F30E94D61C882391F30E94F11F0E94E6
:103F20000707EDCF0C943F1D089508950C94981F3A
:103F3000292F332723303105C9F060F421303105B2
:103F400081F02230310509F044C08BE390E022E893
:103F500032E043C021323105E1F02232310549F12E
:103F600038C082E190E02DEB32E037C099278130F4
:103F7000910549F028F0029761F5E8E5F2E005C007
:103F8000EEE7F2E002C0EEE6F2E0849190E09F01FD
:103F900024C06115710541F061307105D1F489E0EB
:103FA00090E02DEA32E019C089E090E024E932E0A7
:103FB00014C06115710541F06130710551F48BE752
:103FC00090E02FEC32E009C080E490E02AE433E096
:103FD00004C080E090E020E030E0FA0131832083EB
:103FE000089580E189BD82E189BD09B400FEFDCF5D
:103FF0008091D8008F7D8093D8008091E00082600E
:104000008093E0008091E00081FDFCCF0895CF9285
:10401000DF92EF92FF920F931F93CF93DF93EC0108
:104020008B017A010E946521811133C0E114F104F2
:1040300039F0F70180819181081B190BC80FD91F36
:10404000C12CD12C0115110519F18091E80085FDD5
:1040500016C08091E8008E778093E800E114F104A7
:1040600049F0F70180819181C80ED91ED182C082AA
:1040700085E00FC00E946521882321F30AC0899141
:104080008093F10001501109FFEFCF1ADF0ADACF58
:1040900080E0DF91CF911F910F91FF90EF90DF9023
:1040A000CF900895209196023091970226173707F6
:1040B00048F06115710539F42091E8002E772093BE
:1040C000E80001C0B901FC0120E06115710579F13A
:1040D00080918F028823F1F18530F1F18091E80021
:1040E00083FD3CC08091E80082FD2EC08091E800F5
:1040F00080FFEBCF2091F3008091F20090E0922BB3
:104100006115710551F08830910538F421912093A3
:10411000F100615071090196F3CF21E0089709F091
:1041200020E08091E8008E778093E800CECF2111C7
:10413000CFCF0AC080918F02882361F0853061F073
:104140008091E80083FD0AC08091E80082FFF2CFF1
:1041500080E0089582E0089583E0089581E0089565
:1041600020919602309197022617370748F0611583
:10417000710539F42091E8002E772093E80001C002
:10418000B901FC0120E06115710591F180918F0268
:10419000882309F440C0853009F43FC08091E800CD
:1041A00083FD3DC08091E80082FD2FC08091E80032
:1041B00080FFE9CF2091F3008091F20090E0922BF4
:1041C0006115710559F08830910540F424912093D0
:1041D000F1003196615071090196F2CF21E0089704
:1041E00009F020E08091E8008E778093E800CBCF43
:1041F0002111CCCF0AC080918F02882361F08530D5
:1042000061F08091E80083FD0AC08091E80082FFA0
:10421000F2CF80E0089582E0089583E0089581E080
:104220000895982F973068F59093E900981739F022
:104230007091EC002091ED005091F00003C0242F0C
:10424000762F50E021FD02C09F5FECCF3091EB0054
:104250003E7F3093EB003091ED003D7F3093ED00D9
:104260003091EB0031603093EB007093EC002093C1
:10427000ED005093F0002091EE0027FDE5CF80E0A7
:1042800008958F708093E90081E0089580919002F5
:1042900087FF11C08091E80082FD05C080918F02E8
:1042A0008111F8CF11C08091E8008B770BC080910D
:1042B0008F02882349F08091E80080FFF8CF809139
:1042C000E8008E778093E80008952091E400309113
:1042D000E50095E64091EC00842F817040FF23C0FB
:1042E0008091E80080FD1DC080918F02882399F0A5
:1042F000853099F08091EB0085FD11C04091E4007C
:104300005091E5002417350729F3915011F09A01D7
:10431000E1CF84E0089582E0089583E0089581E08C
:10432000089580E008954091E80042FFDDCF0895B0
:104330000E9406220E940E22E0EEF0E08081816061
:104340008083E8EDF0E080818F77808319BCA7ED52
:10435000B0E08C918E7F8C9380818F7E80831092D1
:104360008E0208950F931F93CF93DF930E9406222E
:104370000E940E22C8EDD0E088818F7788838881E3
:104380008068888388818F7D888319BC10928F0212
:1043900010928B0210928D0210928C0200EE10E0AF
:1043A000F80180818B7F808388818160888342E0EF
:1043B00060E080E00E941121E1EEF0E080818E7FDC
:1043C0008083E2EEF0E0808181608083808188607C
:1043D0008083F80180818E7F8083888180618883DB
:1043E000DF91CF911F910F910895E8EDF0E080816A
:1043F0008F7E8083E7EDF0E080818160808384E0C0
:1044000082BF81E080938E020C94B221E8EDF0E04F
:1044100080818E7F80831092E20008951092DA00EE
:104420001092E10008951F920F920FB60F9211247F
:104430002F933F934F935F936F937F938F939F93AC
:10444000AF93BF93EF93FF938091E10082FF0BC086
:104450008091E20082FF07C08091E1008B7F809312
:10446000E1000E9489248091DA0080FF1FC08091C2
:10447000D80080FF1BC08091DA008E7F8093DA0025
:104480008091D90080FF0DC080E189BD82E189BDA6
:1044900009B400FEFDCF81E080938F020E945B1E75
:1044A00005C019BC10928F020E94691E8091E10024
:1044B00080FF19C08091E20080FF15C08091E2006A
:1044C0008E7F8093E2008091E20080618093E20021
:1044D0008091D80080628093D80019BC85E08093D9
:1044E0008F020E946E1E8091E10084FF30C0809197
:1044F000E20084FF2CC080E189BD82E189BD09B45E
:1045000000FEFDCF8091D8008F7D8093D8008091F0
:10451000E1008F7E8093E1008091E2008F7E8093A6
:10452000E2008091E20081608093E20080918B0242
:10453000882311F084E007C08091E30087FD02C06A
:1045400081E001C083E080938F020E94761E8091FB
:10455000E10083FF29C08091E20083FF25C08091A4
:10456000E100877F8093E10082E080938F021092C8
:104570008B028091E1008E7F8093E1008091E200C8
:104580008E7F8093E2008091E20080618093E20060
:1045900042E060E080E00E9411218091F00088609C
:1045A0008093F0000E946C1EFF91EF91BF91AF913C
:1045B0009F918F917F916F915F914F913F912F913B
:1045C0000F900FBE0F901F9018951F920F920FB66D
:1045D0000F9211242F933F934F935F936F937F9389
:1045E0008F939F93AF93BF93CF93DF93EF93FF93FB
:1045F000C091E900CF708091EC00D82FD17080FD80
:10460000D0E81092E9008091F000877F8093F0005D
:1046100078940E9429231092E9008091F00088602C
:104620008093F000CD2BCF70C093E900FF91EF9104
:10463000DF91CF91BF91AF919F918F917F916F91BA
:104640005F914F913F912F910F900FBE0F901F9050
:1046500018951F93CF93DF93CDB7DEB7AA970FB608
:10466000F894DEBF0FBECDBFE0E9F2E08091F1002B
:10467000819322E0E839F207C9F70E94941E8091E5
:10468000E80083FF2EC18091900290919102492F02
:1046900050E04A30510508F024C1FA01EE59FF4FAD
:1046A0000C94CB24803821F0823809F01AC108C05C
:1046B00080918C0290918D02992389F082600FC0C5
:1046C000809194028F70873008F00BC18093E900CD
:1046D0008091EB0085FB882780F91092E90090918A
:1046E000E800977F9093E8008093F1001092F1002A
:1046F000D1C0282F2D7F09F0F4C0882319F0823013
:1047000061F0EFC080919202813009F0EAC09330ED
:1047100009F080E080938D022EC080919202811179
:104720002AC0809194028F702FEF280F263008F056
:10473000D8C08093E9002091EB0020FF1CC093308B
:1047400021F48091EB00806214C09091EB009061A5
:104750009093EB0021E030E0A90102C0440F551F07
:104760008A95E2F74093EA001092EA008091EB000C
:1047700088608093EB001092E9008091E800877FC9
:104780008093E8000E944621ACC08111AAC010911C
:1047900092021F778091E3008078812B8093E30061
:1047A0008091E800877F8093E8000E9446218091F5
:1047B000E80080FFFCCF8091E30080688093E300F5
:1047C000111102C082E001C083E080938F0289C092
:1047D0008058823008F085C08091920290919302B7
:1047E0008C3D53E0950779F583E08A838AE28983DB
:1047F0004FB7F894DE01139620E03EE051E2E32F3C
:10480000F0E050935700E49120FF03C0E295EF7071
:104810003F5FEF708E2F90E0EA3010F0C79601C036
:10482000C0968D939D932F5F243149F74FBF8091A0
:10483000E800877F8093E8006AE270E0CE0101968D
:104840000E94522016C06091940270919502AE01B0
:104850004F5F5F4F0E94961FBC01892B09F441C036
:104860009091E800977F9093E80089819A810E9457
:10487000B0208091E8008B778093E80032C08038C8
:1048800081F58091E800877F8093E80080918B021A
:104890008093F1008091E8008E7772CF811121C062
:1048A000809192029091930299270297D4F480917B
:1048B000E800877F8093E8008091920280938B02CA
:1048C0000E94462180918B02811106C08091E300F5
:1048D00087FD02C081E001C084E080938F020E94C6
:1048E000801E8091E80083FF0AC08091E800877FE6
:1048F0008093E8008091EB0080628093EB00AA96A1
:104900000FB6F894DEBF0FBECDBFDF91CF911F91E0
:1049100008950895CF9380918F028823A1F0C091CC
:10492000E900CF709091EC00892F817090FD80E8B4
:10493000C82B1092E9008091E80083FD0E94292392
:10494000CF70C093E900CF9108950E9498211092F2
:104950008F020895E8EDF0E08081806180838AE134
:104960008A95F1F700C08091D9008170089597FB76
:10497000072E16F4009407D077FD09D00E94D124A9
:1049800007FC05D03EF4909581959F4F0895709552
:1049900061957F4F0895EE0FFF1F0590F491E02D74
:1049A0000994AA1BBB1B51E107C0AA1FBB1FA61776
:1049B000B70710F0A61BB70B881F991F5A95A9F7C8
:1049C00080959095BC01CD010895FB01DC0104C0E8
:1049D0008D910190801921F441505040C8F7881BF7
:1049E000990B0895FB01DC0102C001900D9241502A
:1049F0005040D8F70895F999FECF92BD81BDF89A3D
:104A0000992780B50895A8E1B0E042E050E00C9409
:104A10002F25262FF999FECF92BD81BDF89A0197D7
:104A200000B4021639F01FBA20BD0FB6F894FA9AF6
:104A3000F99A0FBE08950396272F0E940A250E9417
:104A40000925252F0E940A25242F0C940A2501965A
:104A5000272F0E940A250C940925DC01CB01FC01BB
:104A6000F999FECF06C0F2BDE1BDF89A319600B4C7
:0E4A70000D9241505040B8F70895F894FFCFD2
:104A7E00C8000C0201000000010000000000000050
:104A8E00040100000004050000000000002808508A
:104A9E00011E0A1401D91DFC1DDD1D571E531EDCFF
:104AAE001D01E200E900EA00B500B600B700CD0036
:104ABE008301CC008A019201940121022302240277
:104ACE002502260227022A02B300B4006F007000EE
:104ADE00818283E200E900EA00B500B600B700CD9E
:104AEE00008301CC008A0192019401210223022449
:104AFE00022502260227022A02B300B4006F0070BC
:104B0E0000818283F4F5F6F73133946697C62F024F
:00000001FF
